:040000008601772CD2
:08000800A000030E8312A10009
:100010000A08A2008A01931F42288C10131C2C2866
:100020001F151E08FC3CFC3003181E08931E990087
:10003000B600AC17931C2528061CFB3E0618053E8F
:100040005502FE30031CFD30860022088A00210E76
:100050008300A00E200E0900D60803192528D60318
:100060000408D70055088400000ECF389700800C94
:10007000000C3F39950057088400A130D50A0319B8
:10008000D50025280B1E4A288B100B120F3090002C
:10009000B716C0150C104816370B4812C030481E52
:1000A000FE308F001415240BA400250B64002030B3
:1000B000481E0130CB02031D25284B179414C10A9A
:1000C00041083C3C031DC428C101250BA5001F307D
:1000D000A505370BB700C20A421C7028370BCB03AB
:1000E00042083C3C031DA628C2010730481A400BB9
:1000F000C000C30A4308183C031DA628C3011414FA
:10010000BA0C7E30BA050319BA17BB0A1F30BC1DE2
:100110008C283C1C013E95283C188A283C199528BF
:10012000BD0803391D3003191E303B02031CA628ED
:10013000BB01BB0ABC0A0D303C02031DA628BC0152
:10014000BC0ABD0A3D08643C0319BD000408A300B5
:100150002D308400001CBB2800083A050319BB2879
:10016000840A00084202031DBC28840A00084302D6
:1001700003198017BD28840A840A840A0408363CBF
:10018000031DAA28230884004D0BCD00460BC60092
:10019000C71F2528C40A44083C3C031D2528C40168
:1001A000C50A25280530F40081309F0083160D30E4
:1001B000D400E33084001830D500D60112238A1110
:1001C000E4308400C71A800E85120B13A201970138
:1001D0000711F201F3018030DA00D6006430D80054
:1001E000831653309200831214309200BB22D60B38
:1001F000F6280B139722D900D5013930D6005A08BA
:100200009E00BE221F151E08C71999005902031827
:10021000D9021E085502031CD5025A081E02D3003B
:100220000310DD19D30D530D5D1AD30C530DDD1AD8
:10023000D30C530D5D1BD30C530DDD1BD30C0F30B2
:10024000D30507308A002130DE07F0305E05530405
:10025000FF26D4000F39D419F038E407540E0F39B3
:10026000D41BF038E5072A30DF07F0305F05530470
:10027000FF26D4000F39D419F038E607540E0F3991
:10028000D41BF038E7073430E007F0306005530442
:10029000FF26D4000F39D419F038E807540E0F396F
:1002A000D41BF038E9073D30E107F0306105530415
:1002B000FF26D4000F39D419F038EA07540E0F394D
:1002C000D41BF038EB074630E207F03062055304E8
:1002D000FF26D4000F39D419F038EC07540E0F392B
:1002E000D41BF038ED074F30E307F03063055304BB
:1002F000FF26D4000F39D419F038EE07540E0F3909
:10030000D41BF038EF07D60B01290B175908D5027B
:100310000310D50C5507DA005508023CDD0C0630F9
:100320005502DD0C0C305502DD0C17305502DD0C8A
:100330002D305502DD0C643084000008003C801B29
:100340008000000DD9000301D90D03180007800CAF
:100350008008031DA429800084038007FF30031850
:100360008000840A840A041E9D29AC225408DC0003
:1003700084008001AC22D405DC055C085402540ED4
:10038000DC040318DC0E0C30D90002308A0059035B
:100390009F225C020319CE29D90BC729BC307307F1
:1003A0008400F3080319DA29000859020319482ABE
:1003B000AC1FDD29840AF30AAC1359088000E5302C
:1003C000840058030002031CF329840A000AAC1BB2
:1003D000000873020318F329840A000884038403C5
:1003E0008000740B592AD80BF92897220A30AC1FC9
:1003F000F3037302031C3F2A013ED400BD30730790
:10040000D500D503550884000008D9000930D6006E
:10041000840200085902031D102AC2220319552A1A
:10042000CA22D40B012ACA22E80803193F2A031062
:10043000680C69078400E9000930D6008402C222F2
:100440005603DC00083CD6000403D50058302707CB
:10045000D400D80086225C08D6006903D500862225
:1004600058088400D61500080C3C590E031980006A
:10047000000ED900840AD60B332A2708DE00121199
:10048000AC10DE08031DF92BDE0A0F30DF00F92B5C
:1004900059080319DF29AC1BDF29AC177202031DB1
:1004A000532AF303DF29F202DF29E60A5508E700A1
:1004B000112AF4000B138316AC3092008312E33040
:1004C00084000008D600840A800D0C30031C3C30E8
:1004D0009200970103189709E8300318822AA61A98
:1004E00087120711BB228716A61A0715BB22D60B47
:1004F0006F2AE428A61E970100089500BB22840AF3
:10050000041E7A2A8400D60B7A2AE428D608031916
:1005100008008E22D503D40AD603872A5508840002
:100520000008D90054088400590880000800DE0142
:100530005F3084008001840A041E9A2AFF348207F7
:100540004634483468344A346A348A344C346C341F
:100550008C34AC348E34AE3464308400D50155080C
:100560000002031CB62AD5070408D400840A840AB2
:10057000041EAF2A0F340C184A2083128C1CBE2A8A
:100580008C10E8340B30000203190800840FD60BDE
:10059000C22A0800660868020318D12AE802670820
:1005A000E900E60108008312071200008711831694
:1005B000560D0F39A0388312DD000830DC00DD1B3A
:1005C0000716DD0D8715000087110712DC0BDF2AE7
:1005D00083160716831287158310071A8314871151
:1005E0000712831607120134723084000930831613
:1005F000D400D501D601012B8316D400D6010408FE
:10060000D5000310D322831C072B3C23012B550854
:10061000DB220009DB22D5070318D60A840AD40B93
:10062000052B3B2B0310D322831C182B3C23122BAE
:100630005508DB228312071687150314D32283166D
:1006400007168312DC1587150310071A0314871188
:10065000DD0DDC0B232B5D098000840A0712831655
:100660000712D4038312031907168715372B871136
:10067000031D1F2B07128A1583128715000007160A
:100680000134FF300C1E422B990008000830A400F2
:1006900083148C1A4E2B240B492B552B8310981C3A
:1006A000542B1812831418161A08CC008318C81774
:1006B00003140800FF30D8004123580A0319072CFF
:1006C0004223581F6D2B5E3084000008FE00FE0A96
:1006D0004223840A0008FE0B682B8A150034462347
:1006E0008318582BB6231318992BA130D500D400AA
:1006F00011309900A42303188B2B5608323C0318A1
:100700007A2B13309900A42303188B2B1630560232
:10071000031C782B832B8316A40183160B138C10D8
:100720000C148312920193010B179701C601031059
:100730007D340A30A400CF23240B9B2B8C1A8B2BE7
:100740008A1503238A119E2B8C1EB22B5408840019
:100750001A088000D60A013E03180800A130D40A06
:100760000319D4000C184A208312972B0B13930003
:10077000D60113188512131C85169F179F111F127F
:100780009F1213181F148716970183163C3092008E
:100790000C108C148312143092000B1708003C309C
:1007A000D8008A15742174218A11AC133608D3003D
:1007B000DB008A1503238E218A1136080318DB001B
:1007C0005302031CD302D80BD92B5B08D3020310AE
:1007D000530C5B07D500DB00080083128C1AFD2B3D
:1007E0008314460BF92B4030CC0083102030C60018
:1007F0004C088A1508008314F92BB7164E232C19C0
:10080000032C2C15FB2B031D0D2C4123412C4C08D4
:1008100080384223462383186D2BCC1FF52B4C1CAC
:10082000142CB930AC05FB2BDA004223DA1C212C46
:100830004623C81B412C84002130031D000842239D
:10084000412C5A1D292C462384004623C81F8000B2
:10085000412CCC1D3A2C47240B1F1D238A11C81B89
:10086000412C84034C0842238316D40A8312DB0BE9
:100870002D2C412C4C1E3F2C49248A11412C4C1B01
:100880006F23C813AC1CFB2B8C1AED2B442C462376
:10089000DB00D6308400462380008403462380009A
:1008A0008403013080004C30840083165608073CD6
:1008B000031C632C8312C81B0134DA19122B462344
:1008C000C81F012B01340F30D600FC30D504D701EE
:1008D0008312C817DA1D5F2CAE248403D40A0330B8
:1008E000D70583124C084223DB0B6C2C0134831692
:1008F000013086008F308100DF3085008130870035
:100900008C00023099002630980002309F0083123C
:100910008516183087000F309000920197019D01D5
:10092000903098009301DE018316A401031EA92CC8
:100930000630D600D830D50025308400D7011B30D2
:10094000D400AE2483168E18A92C8E140C30D4003B
:10095000AE24C0308B008A158312602C8316B82415
:100960000B178A118000840AD70AD40BAE2C08001A
:1009700056088A00550857070B1303188A0A820085
:100DB0000734703407340134003401340034003413
:100DC0000034003400340034003400340034003483
:100DD0000034003410348A34253480340934033428
:100DE0006234003400340734003400340C340034EE
:100DF00000342034003400340134013440348200A3
:100E000000341034203430344034403450346034B2
:100E10009034A034B034C034C034D034E034F03432
:100E200000341034213421343134423452346234A9
:100E30009D34AE34BE34CE34DF34EF34EF34F0348E
:100E400000341134113422343334333444344434D0
:100E5000BB34CC34CC34DD34DD34EE34FF34FF34F9
:100E6000003401341234123413342434253426343B
:100E7000D934EA34EB34EC34FD34FE34FE340F3430
:100E800000340134023403340434043405340634A9
:100E900009340A340B340C340C340D340E340F3452
:100EA00000340134F234F234F334E434E534E6341B
:100EB00039342A342B342C341D341E341E340F3470
:100EC0000034F134F134E234D334D334C434C43490
:100ED0005B344C344C343D343D342E341F341F3499
:100EE0000034F034E134E134D134C234B234A234C9
:100EF0007D346E345E344E343F342F342F3410340E
:100F00000034F034E034D034C034C034B034A034D1
:100F10007034603450344034403430342034103431
:100F20000034F034EF34EF34DF34CE34BE34AE343A
:100F30007334623452344234313421342134103425
:100F40000034FF34FF34EE34DD34DD34CC34CC34C3
:100F5000553444344434333433342234113411346A
:100F600000340F34FE34FE34FD34EC34EB34EA3418
:100F700037342634253424341334123412340134F3
:100F800000340F340E340D340C340C340B340A346A
:100F90000734063405340434043403340234013491
:100FA00000340F341E341E341D342C342B342A34B8
:100FB000D734E634E534E434F334F234F234013433
:100FC00000341F341F342E343D343D344C344C3403
:100FD000B534C434C434D334D334E234F134F134CA
:100FE000003410342F342F343F344E345E346E349A
:100FF0009334A234B234C234D134E134E134F03425
:101000005E0A0F3C0318DE0A5E305E0784000800AB
:101010008316180983122C040639031963008A11F8
:10102000031E00288A15031D9922400B21289001D8
:101030009F018B100B1663000000031E1B288A11F2
:10104000002806221F30C805C71B782846214621E4
:1010500046213621490BC6283D214A0B9B285308BF
:10106000013C031CB71603189B28DE01C222C130C5
:10107000842146234122DD01862144080F3CB430FF
:10108000031C1D2AC420062286212F2103183B2879
:10109000261E7328C8197328D6018621D60A561E23
:1010A0004D282F21031862288621D60AD61F5128E1
:1010B000C71B7A23F9222F24C701B330842146218C
:1010C00093229B285608283C03183B28DD0AD601AA
:1010D00086212F21031C4828D60A561F6828002085
:1010E0005D08800037284D2193224621C2224C28DA
:1010F0002C1A5F28AC199A282F21031883288721DE
:101100002F21031C5A285308013C031C8D28510B26
:10111000D100FF3903195A289B28D115083E031C1A
:1011200094284F0FCF009B28CF1B98284F1B0A2BCA
:10113000F9229B284D21410BB928420BB928941C58
:10114000B92889309F000C1EA328992200309900ED
:10115000BA3081000B110B1DAB281F151F19AE28CB
:101160001E08763C83160318A4168312BB3003189E
:10117000842194101F100301AF1B532C013EB21B9E
:10118000532C013EB51B532C8A11ED2BFF38261B27
:1011900028080319EA28D7000730CD003D23CA00EC
:1011A000D7030319E628C420AC19EA282C1AE22830
:1011B0003521490BCC283D214A030319E9284D0B61
:1011C000D3285F284D219322EE225F281A309422E3
:1011D000EA28C7164D218A11D220C030842142232B
:1011E0001F30A61A9422C71AF728AC19F7287821BD
:1011F000031827292E232F23782103182729831644
:10120000CA30920083127F309200033095003F3045
:10121000970033309422970112117821031827295F
:101220009630A400CF01782103182729C420AC19D7
:1012300025292C1AE428A130C7210318CF0A4F19F9
:10124000E428240B1629EE22F728EE225E2CC7167E
:101250005E2C1F151F192A291E08D30008002921FA
:10126000390221342921093C08008621292138022C
:10127000031CC916490BC900080053083902403045
:1012800003184A0BCA00031CB716080085169930CC
:1012900087002C12AC11D83407150130CA0087160C
:1012A000D8348512D83485163C340310AC190800A4
:1012B000D108031908000F304F05031D080047210E
:1012C000062274217421FE01AC1F6429AC13360878
:1012D0003902031C7029FE0B642981309F00832989
:1012E00081309F004D217421AC13AC1F752908007B
:1012F0000310481B080046210622FE012F21031C73
:101300004D29FE0B7E29B9308A115B2B0730FE0078
:101310000B110B1D8929FE0B88296C34AC1F8E29FB
:10132000AC1336085B0203080139080002305A1C6E
:10133000FE30DB078E215A06031DA029D60B9A2901
:10134000FE00DA06FE305A1C02307E18003CDB0735
:101350003F340C1CA92903238E21DA001E30D6004D
:1013600096217E1C3F341E30D60096217E1C3F34D1
:1013700096217E1856080800D900143C1F30031C23
:10138000C52959085302031C003CD40708008A11E0
:10139000B623CF238A15D301D401D814A921D307AA
:1013A000B121D307D80BCE295815D30C530C3F3994
:1013B000D300A921BC21B121BC21D80BD9295408C3
:1013C000113C0800CF0AC7210318F4290323D10ACE
:1013D00050080319F129D001053C0434D20103144B
:1013E000003451084E0201340323D00A500B042A62
:1013F0005108D101083C031CEE29063C031CEE29D0
:10140000D20A5208023C0234163C083499309F003C
:101410004B34C71B602CCD01482341225B220318AB
:10142000142AC822031C1F2AFF3903191B2ABA30A9
:1014300084214D0B0E2A4621B53084215D2CB43019
:1014400084217A23C71E262AEE22602CAC19242A76
:10145000C4202C1E2D2A4621242AAC19242A83308C
:10146000481DA130E2210318392AD900F922D918E0
:101470002B2A5521C712031C3F2AC716242A0323EF
:10148000282A47135E308400000803190800DD0095
:10149000840A00080F3C031D502ADD0B482A08006F
:1014A000F93E031D080047175D0B0800DE0A840A99
:1014B0000F308000080046210622DC0099222921F5
:1014C0003D21DC0B5E2A4A08013C031800344D2103
:1014D0009322F922C4202C1E702AEE220314003419
:1014E000A130E221031C782A4F1F782AEE22003413
:1014F000D01D6A2AEE225F30F0005E08DC00013C5D
:101500000318003470088400F00A0008CC009D2203
:1015100003180800C42003142C1A0034DC0B822AA0
:10152000CE300310942A41308312A400240B962A53
:1015300008001411141D9A2A08004C080B3C031CC7
:10154000B22A0319C816FF30C81A842930309422F1
:101550004621872187214C218721CC0BA82A0711FE
:1015600003100800043E031DEF29F9228330481DB3
:10157000A130E221031CC02A4F1FB62AEE220234FA
:10158000073CBE2AC713C52AC717C401C501EF29E6
:10159000F922CE003C30C600C422C4202C1A6D2A89
:1015A000AC19B02A8330481DA130E2210318E62A85
:1015B000D900F922591DE02A4C1FCC2AEE22C22A5A
:1015C0005918B02AC222EE22031402345521C7163C
:1015D0000318B02AC7124F0FCD2AB02A83160B1357
:1015E0008C100C1483129701920193010B170711B1
:1015F0008516C8124630CE00CF01D001D201093085
:10160000D1008314FD340C1C08008A114A208A156D
:1016100083120800D001CF018621322103181F2B2D
:10162000CF0ACF1F0C2B50080319F92A2A02031DD9
:10163000F92A4817C7124D21B2308421F7284F08E4
:10164000283C0318F92AD00ACF0186213221031C35
:101650000B2BCF0A4F1F252BF92A08000800323028
:10166000A400240B312B08000B1383168C100C14D0
:101670008312930192010B17542935214903031951
:10168000342B3D2B471647230E307B2BC716C42225
:101690000B134208F2004308F3003B080B17F40059
:1016A0007530D400540884008001840A841F542BB0
:1016B0005E0803190800D8000F3C5E08031C0F30B9
:1016C000DE00D600D60A5E308400000E840AD60BF7
:1016D0000004D900040AD50054088400590E800083
:1016E000D40AD6080319772B5508D60B642B580853
:1016F000DE0008000930B82393238312471A892B90
:10170000F5080319471627087502831C0134C71B07
:10171000C7148316B8308400D40A9123C1237230D1
:1017200084008A11012B83163B08B8030319B80003
:101730000800DE30D400550884000008D6000F30C1
:10174000D605D60A0008D9005408840059080F3974
:101750008000D60BAC2B0800840A590E0F3980008C
:10176000D40AD40AD50A55088400D60BA22B080047
:101770008316D500D6010530D400B83084008A1114
:10178000122B83163808DB003908D6003A08D5003A
:101790003C08D400D5070318D60ADB0BCA2B080077
:1017A0000310DE080319FB2B7330D7001330B82366
:1017B0008316B800C12372308400BF235708D500B8
:1017C00099235E08D60083165E028312031CF42B55
:1017D000DF3084000008841300028417031DF42BFB
:1017E000840AD60BEA2B08008316B80A38083B0295
:1017F00083120318DA2B290803390800D023031CAD
:1018000008005E0883165E02831203190800F423A1
:10181000FF2BFB01831672308400D501D6010930FD
:10182000D400BF231D24471B753084007B0880072C
:1018300084030318800A8A11F42A3C08FA02FA0089
:10184000031973347208F201F6007308F301F7000C
:101850007408F401F8007508F501F9007334471AAB
:101860000134C7134508031D392C44080A3C0318EA
:1018700001344408031D01304507FB000A24C71C3E
:1018800001340930B823C123FF3ED5070318D60A17
:101890000130D4007B308400912B56085607560740
:1018A0002A3E84000800B716D600D60AB630842136
:1018B0004D24023E84008013602C7A232030C60021
:1018C0000730A50408208318602C4C1B602C0C3CAE
:0618D0000319092A602C37
:081FF8000034013433340234DB
:00000001FF
